S00A000050332E7372656397
S11300000C9434000C9446000C9446000C94460066
S11300100C9446000C9446000C9446000C94460044
S11300200C9446000C9446000C9446000C94460034
S11300300C9446000C9446000C9456000C94460014
S11300400C9446000C9446000C9446000C94460014
S11300500C9446000C9446000C9446000C94460004
S11300600C9446000C94460011241FBECFEFD8E038
S1130070DEBFCDBF21E0A0E0B1E001C01D92A430FD
S1130080B207E1F70E94B7000C94CC000C94000076
S113009084B5826084BD85B5836085BD89EF87BDE5
S11300A0EEE6F0E080818260808308951F920F92D3
S11300B00FB60F9211248F939F93AF93BF938091A8
S11300C0000190910101A0910201B09103010196F8
S11300D0A11DB11D8093000190930101A093020121
S11300E0B0930301BF91AF919F918F910F900FBE79
S11300F00F901F901895F894609100017091010180
S1130100809102019091030178940895CF92DF9237
S1130110EF92FF926B017C010E947B00C60ED71EFA
S1130120E81EF91E0E947B00C616D706E806F906EB
S1130130C9F7FF90EF90DF90CF900895CF92DF92B0
S1130140EF92FF926B017C010E947B006C157D0590
S11301508E059F05C9F7FF90EF90DF90CF9008952B
S1130160509A08959BB181E089278BB908950E9424
S1130170B0000E94480064EF71E080E090E00E94CB
S11301809E000E94B20064EF71E080E090E00E9463
S10F019086000E94B200F7CFF894FFCF65
S9030000FC
